:102000003C00680074006D006C003E000D000A008A
:102010003C0062006F0064007900200062006700ED
:1020200063006F006C006F0072003D00220023000F
:1020300039003900390039003900390022003E00EA
:102040000D000A003C006400690076002000610079
:102050006C00690067006E003D00220063006500AF
:102060006E0074006500720022003E000D000A0040
:10207000200020003C007000200061006C0069001E
:1020800067006E003D002200630065006E00740072
:102090006500720022003E003C0066006F006E008A
:1020A0007400200063006F006C006F0072003D0040
:1020B0002200230046004600460046004600460037
:1020C00022002000730069007A0065003D002200B4
:1020D00037002200200066006100630065003D00BB
:1020E0002200560065007200640061006E0061000D
:1020F0002C00200041007200690061006C002C007F
:102100002000480065006C007600650074006900DE
:10211000630061002C002000730061006E007300FA
:102120002D007300650072006900660022003E0009
:102130003C007300740072006F006E0067003E0088
:102140005000690063006F00490050003C002F0000
:102150007300740072006F006E0067003E003C0068
:102160002F0066006F006E0074003E003C002F00E0
:1021700070003E000D000A00200020003C007000AE
:10218000200061006C00690067006E003D002200C5
:10219000630065006E0074006500720022003E005E
:1021A00026006E006200730070003B003C002F00B0
:1021B00070003E000D000A003C00680072003E0006
:1021C0000D000A003C0070003E003C0066006F00FD
:1021D0006E007400200063006F006C006F007200DE
:1021E0003D0022002300460046004600460046000F
:1021F000460022002000730069007A0065003D005F
:1022000022003200220020006600610063006500A9
:102210003D002200560065007200640061006E00FF
:1022200061002C00200041007200690061006C0018
:102230002C002000480065006C00760065007400EA
:102240006900630061002C002000730061006E00D3
:1022500073002D00730065007200690066002200A3
:102260003E004200690065006E00760065006E0069
:10227000750065000D000A007300750072002000F3
:102280005000690063006F00490050002C002000DE
:102290006C006500200070006C0075007300200069
:1022A0007000650074006900740020007300650010
:1022B00072007600650075007200200077006500EE
:1022C000620020006F00700026006500610063005E
:1022D0007500740065003B007200610074006900C5
:1022E0006F006E006E0065006C002000320034004C
:1022F00048002F003200340048003C002F006600E8
:102300006F006E0074003E003C002F0070003E0025
:102310000D000A00200020003C0070003E00260056
:102320006E006200730070003B003C002F007000E4
:102330003E000D000A00200020003C0070003E001E
:1023400026006E006200730070003B003C002F000E
:1023500070003E000D000A00200020003C007000CC
:102360003E0026006E006200730070003B003C00DF
:102370002F0070003E000D000A003C002F0064009A
:10238000690076003E000D000A003C002F0062004C
:102390006F00640079003E000D000A003C002F0031
:00000001FF
